:020000040000FA
:100000001C28C501051801280830C600E120E4209D
:100010000314051C0310C50CE4200000C60B0828BF
:100020000800113084001A30B40001204508800017
:10003000840AB40B15280800830185018601831604
:10004000013085008601831285011A308600012067
:1000500045085A3C031D272801204508443C031D40
:10006000272801204508413C031D27280120450879
:100070002C3C031D272811203E2024288A30B9005B
:1000800016080F39103EB70086000030B800850012
:10009000DB2015080F39103EB70086000230B8008B
:1000A0008500DB2014080F39103EB70086000630AB
:1000B000B8008500DB2013080F39103EB70086001A
:1000C0000830B8008500DB2012080F39103EB70059
:1000D00086000C30B8008500DB2011080F39103E77
:1000E000B70086000E30B8008500DB20B90B402831
:1000F00008008A30B90024080F39103EB700860086
:100100000030B8008500DB2023080F39103EB7000F
:1001100086000230B8008500DB201F080F39103E32
:10012000B70086000630B8008500DB201E080F39B6
:10013000103EB70086000830B8008500DB201C08A0
:100140000F39103EB70086000C30B8008500DB2068
:100150001B080F39103EB70086000E30B80085002E
:10016000DB20B90B402808001430B400BA20B40BCF
:10017000B62808006230B1006430B200B20BBE286D
:10018000B10BBC2808001230B1002130B200B20B14
:10019000C728B10BC52808002230B100B10BCE280A
:1001A00008006830C200C20BD3280800C300D12069
:1001B000C30BD72808000330C400D120C40BDD28AE
:1001C00008001530C700E7284130C7000000C70B02
:0401D000E728080014
:02400E00F13F80
:00000001FF
